:020000020000FC
:100000000C947D095BC200000000000000000000AD
:1000100000000000000000000000000000000000E0
:100020000000000031C00000000000005DC10000C1
:1000300000000000000000000000000000000000C0
:1000400059C1000000000000000000000000000096
:100050000000000002030406080C10182030406065
:10006000800002030406080C101820304080FF00B6
:100070000406080C10182030406080A0C000050560
:100080000D050D06020303024FB662FD22C070FF8C
:100090001DC165FDFDC057FE01C00994C091370127
:1000A000C395C0933701C5E0C519B8F3D0913701A6
:1000B000CD1B98F3C8E7089483FDC795C093B200A1
:1000C000C52DCC2329F4C0E083FDC0E8C093B20065
:1000D00009C171FF03C02B982C982D98C52D089449
:1000E00083FDC795C093B200C09339016B7FC52DC6
:1000F000CF3F09F441C0C0913801C395C093380186
:1001000070FF35C02B982C982D984FBE18957860AD
:10011000C0914001CC2391F0C0913801CA95D09193
:100120004001CD1B58F0777FC0913801D0913F013D
:10013000CD1B08F41CC02092380119C02B982C98B4
:100140002D98C1E0CA95F1F7C0911501CA95C2FD7D
:1001500009C0C1FD05C095FF299A95FD2A9A0EC0D8
:10016000289A0CC095FF2A9A95FD299A07C02B98CA
:100170002C982D984FBE1895209239014FBE189596
:10018000A5C0552021F095FF2B9A95FD2D9A2C980E
:100190009DC0552009F02C9A95FF2D9895FD2B9820
:1001A00095C0552021F095FF2D9A95FD2B9A95FF2E
:1001B0002B9895FD2D988AC095FF2A9895FD299832
:1001C00095FF299895FD2A98C1E0CA95F1F7552029
:1001D00021F095FF2B9A95FD2D9A2C9877C095FFCD
:1001E0002A9895FD29982898C1E0CA95F1F75520DD
:1001F00021F095FF2B9A95FD2D9A2C9867C0289891
:1002000095FF2A9895FD2998C1E0CA95F1F75520E8
:1002100009F02C9A95FF2D9895FD2B9857C028989A
:1002200095FF299895FD2A98C1E0CA95F1F75520C8
:1002300009F02C9A95FF2D9895FD2B9847C095FFB6
:10024000299895FD2A982898C1E0CA95F1F755207C
:1002500021F095FF2D9A95FD2B9A95FF2B9895FDF2
:100260002D9834C095FF299895FD2A9895FF2A98D6
:1002700095FD2998C1E0CA95F1F7552021F095FF29
:100280002D9A95FD2B9A95FF2B9895FD2D981EC0C4
:1002900082FF1CC0C0911501C2FD0BC0C1FD11C081
:1002A00095FF2A9895FD299895FF299895FD2A98FC
:1002B0000DC0C1FDF5CF95FF2A9895FD2998289886
:1002C00005C0289895FF299895FD2A98C52DC095B9
:1002D000089483FDC795C093B200C0933901209262
:1002E000370164604FBE18954FB6C2E0C6BB6E7F43
:1002F0004FBE18953FB68F7EADB3A170A21180613D
:10030000A0E0ADBBA0916E00AE7FA0936E0078948C
:10031000A0910601AA2349F0A92FAF7159F1A0912C
:100320000601AA95A093060125C040E050E0A9B1BE
:1003300096FDA095A2FD4FEF96FFA3E096FDA2E0EB
:10034000A0936900AA27A160ACBB8D7FA9B196FDDF
:10035000A095A2FD5FEF451741F7A8E161FDA093CD
:100360000601A92FAF7119F0A8E1A09306014093EF
:100370002D018160A0910701AA2331F0A09107010E
:10038000AA95A093070107C0A92FAF7121F0806142
:10039000AA27A160ACBB80FF48C0A0912D014A2FC5
:1003A0008E7FA92FAF71C1F0403F08F040EFA42F1E
:1003B000A295AF704A0F50915001533069F0A69545
:1003C000A69550FD01C0A69552FD03C0A41B4A2F5F
:1003D00003C04A0F08F44FEFA09136014A1708F402
:1003E0004A2F4093010171FF08C0A0910101509173
:1003F0003201A51710F050930101A0910101409125
:100400000301A41B70F040916F01A40B50F0A09168
:100410000301A40FA093030140F4AFEFA0930301E5
:1004200004C0A0910101A093030140910301A09198
:1004300032014A1708F04A2F542EA52DA03408F097
:100440006860A0910001A395A093000161F0F89469
:10045000A0916E00A160A0936E0084FF02C0A1E095
:10046000ADBB3FBE189541E050910601552331F0D8
:10047000A92FAF7119F45A9550930601A0912D013F
:10048000A13018F0209230010DC02092310120924D
:100490003A01A0913001AF5FA093300118F0AFEFA7
:1004A000A0933001F894A0916E00A160A0936E001B
:1004B00084FF02C0A1E0ADBB3FBE18953FB640919E
:1004C0008400509185008F7EADB3A170A211806130
:1004D000A0E0ADBBA0916E00AE7FA0936E007894BB
:1004E00081FD28C096FFA2E096FDA3E0A0936900DD
:1004F0008260A9B196FDA095A2FF05C040930401BA
:100500005093050136C196FFA3E096FDA2E0A093AB
:100510006900AA27A160ACBB8D7FA92FAF7109F438
:1005200019C140E0A9B196FDA095A2FD13C1409369
:100530002D0106C196FFA3E096FDA2E0A0936900FD
:100540008D7F61FF6CC096FFA2E096FDA3E0A093B3
:100550006900AA27A160ACBB826040932801509338
:100560002901A09026014A19B09027015B09BB24FC
:10057000A2E0EA2EA22C483CA0E05A0730F4A0E109
:10058000BA2EE22CAAE0AA2E27C04836A1E05A07CC
:1005900030F4A8E0BA2EE22CAFE0AA2E1DC0403DF8
:1005A000A2E05A0730F4A4E0BA2EE22CAEE1AA2E63
:1005B00013C0403AA5E05A0730F4A2E0BA2EE22C6C
:1005C000ACE3AA2E09C04839A8E05A0728F4A1E0F4
:1005D000BA2EE22CA8E7AA2EC42EA0912A01CA1A8C
:1005E000D52EA0912B01DA0ADD202AF4AFEFC094BA
:1005F000D094CA1ADA0A20922C01CA14DE0418F424
:10060000A1E0A0932C0140932A0150932B0140912B
:100610002801509129014093260150932701A09170
:1006200004014A1BA09105015A0B94FD7CC093FD67
:100630007AC092FD76C05695479591FD72C0569549
:10064000479590FD6EC0D52EC42ED694C79461FDFB
:100650000CC0AC2DAC51AD2DA24008F07BC0DD200C
:1006600021F4AC2DA85C08F475C0A0E0EA2E97FD3B
:1006700008C0E0906201A0915401A33011F4E09011
:100680006A01AAEFEA0EF22CF21CCE18DF084FB76F
:100690004170A0915401A330A9F4442329F095FDA1
:1006A00011C0F894906204C095FF0CC0F8949F7D2F
:1006B0002B982C982D982A982898299871FD01C07C
:1006C00060687894442369F0A0915401A33031F418
:1006D000AFEFC094D094CA1ADA0A03C040E050E0E9
:1006E00022C0A0915401A33049F4CC0CDD1CA5E03C
:1006F000CA1AD20818F4A0E0CA2ED22CAFEFCA163C
:10070000D20418F04FEF50E00EC0F0904701CF9C9C
:10071000412D000C441F50E008F012C04FEF50E094
:100720000FC05695479594FF07C0552309F04FEF2A
:10073000A42FA6954A0F521D4F3F520508F04FEFC8
:1007400040932D01816061FF05C0AFE1A095A92311
:10075000AB299A2FA8E1A0930601A92FAF7119F434
:10076000AAE0A093060161FD04C0A92FAF7109F0B2
:100770008F7EA6E0A0930701A92FAF7119F4AAE01C
:10078000A0930701F894A0916E00A160A0936E0061
:1007900084FF02C0A1E0ADBB3FBE189511E00AC0C6
:1007A00013E008C01AE006C01EE104C014E602C04F
:1007B00018EC00C005E1BB27BA95F1F70A95D9F707
:1007C0001A95C1F708952AE338E709C020E33CE809
:1007D00006C02AE234EB03C025E238EC00C0652CE9
:1007E000B1E05B2E12E095FD9F7D95FF9062BB27E7
:1007F0002898BA95F1F7552009F02C9ABA95F1F797
:100800002C98BA95F1F7289ABA95F1F7552021F06E
:1008100095FF2B9A95FD2D9AB0914801BA95F1F765
:1008200095FF2B9895FD2D98B7E8BA95F1F71A9595
:10083000D1F6022FB22FBA95F1F70A95D9F73A956A
:1008400071F62898562C0895221B39E0001F3A951E
:1008500009F40895221F211B18F4210F8894F6CF64
:100860000894F4CF622C722CB0E08894B395221FC8
:10087000331FE0F7379527958894912E802E020B31
:10088000130B10F4192D082D10F4889401C008944E
:10089000661C771CBA9571F7172D062D0895322D19
:1008A00011232AF43A9500951095031B130BF89425
:1008B000029F712C002D129F912C802C7894780C23
:1008C000172D921C292DB4E06B2E269517950795B0
:1008D0006A94D9F7332321F000951095031B130B6D
:1008E0000895089566FF21C0109114011695009196
:1008F00013010795B0911701B01B0B2FB091180190
:10090000B10B1B2F28F40038BFEF1B0740F009C0C4
:100910000F37120508F405C00FE710E002C000E829
:100920001FEF00931C0110931D01089566FF39C04D
:1009300000911C01B09119010B0F10911D01B09194
:100940001A011B1F20E030911D0133230AF42A9560
:10095000B0911B012B1F1AF4203F40F00AC02F302A
:1009600008F407C00FEF1FEF2FE003C000E010E016
:1009700020EF30910301B09132013B1718F433237B
:1009800031F009C0B0911D01BB235AF004C0B091F1
:100990001D01BB2332F40093190110931A01209317
:1009A0001B01089566FF30C020916D0100911C016C
:1009B000000F10911D01111F0E944F0411232AF4F2
:1009C0000038BFEF1B0740F009C00F37120508F4CD
:1009D00005C00FE710E002C000E81FEF002352F04F
:1009E000B0910201B01B0B2F18F0013008F00AC0C3
:1009F00001E008C000950F5FB09102010B0F08F0F5
:100A000001C00FEF00931E01089566FF2EC02091D4
:100A10006E0100911A0110911B010E944F041123D5
:100A20002AF40130BFEF1B0740F009C00F3F120549
:100A300008F405C00FEF10E002C001E01FEF112322
:100A400052F0B0911E01B01B0B2F18F0013008F0CE
:100A50000AC000E008C000950F5FB0911E010B0FA7
:100A600008F001C00FEF0093030108950FEF677FB7
:100A7000B72FB670F1F46860B0911401B83008F087
:100A8000677FB0911401A9F00FEF109114010E943B
:100A90002404F894B09110010B9F112D002D78942F
:100AA000112309F00FEFB09135010B1710F40091ED
:100AB00035010093340108957BC00E94630874FFE0
:100AC000B0E074FDB0E0B06CB0937C00B0917A00FF
:100AD000B068B064B0937A000E94CE0374FFB0E0B7
:100AE00074FDB0E0B06CB0937C00B0917A00B06857
:100AF000B064B0937A00B0917A00B6FDFCCF00915B
:100B0000780010917900B0917A00BF77B0937A00A5
:100B10000E94A90827EE2093430130E0309344015E
:100B2000732E7694622E6694620E731E262D372DD8
:100B30000217130778F080904301B7EEB80DB09319
:100B4000430180904401B0E0B81DB0934401260DEC
:100B5000371DEECF809043019090440110914401E5
:100B6000169500914301079516950795B09143019D
:100B7000B00FB0934101B0914401B11FB093420155
:100B800023E0169507952A95E1F720914F012A95C4
:100B900029F420924301209244010AC02A9521F0B1
:100BA000800E911E2A95E1F78092430190924401B4
:100BB000089520914F01B0917A00B6FDFACF0091CF
:100BC000780010917900B0917A00BF77B0937A00E5
:100BD000B0914501B395B0934501B83060F12092D2
:100BE0004501B0916C01BB2321F1112329F0B09193
:100BF0004601BF3F61F009C0B09146010B1739F0C3
:100C000020F4BB2321F0BA9502C0B395E1F3009123
:100C10003201B0934601B03050F400ECB03038F4FB
:100C200000E8B03020F400E4B03008F400E00093B5
:100C300032017F7E0895B0913201B39511F0B093E7
:100C40003201B0914501B73009F47061089502E3B3
:100C5000F894B09170010B9F012D000C001F789447
:100C6000B09132010B1710F0009132010093010195
:100C700000930301502E0093350108952092130133
:100C8000B8E0B09314010895209120013091210122
:100C9000F8940091840010918500200F311F30934B
:100CA0008900209388006160B2E0B6BB78942091FF
:100CB0001101309112010093110110931201021BD6
:100CC000130B2091130130911401622E732EB4E0A6
:100CD0008B2EB2E09B2EB0911401B43010F08A94A8
:100CE0009A94B83010F08A949A94769467948A947F
:100CF000E1F726193709992021F0169507959A945E
:100D0000E1F7200F311F209313013093140108F0F5
:100D10000895BFEFB0931301B0931401089520918B
:100D2000220130912301F8940091840010918500F4
:100D3000020F131F10938900009388006160B2E0D6
:100D4000B6BB7894089560FDFECF0E948F0608958B
:100D5000B0915E0100910E01023808F0B395003A9F
:100D600008F0B395B63008F0B5E09B2EBCE08B2EB2
:100D7000B0911401B33030F48394839482FF02C0A5
:100D800083948394B23030F48394839482FF02C0BE
:100D90008394839471FF03C0B3E09B2E822C109147
:100DA00014010091130124E0169507952A95E1F7A7
:100DB0000819120928F0B02FB250B12FB20910F45F
:100DC00002E010E0312F202F712E602E7694679470
:100DD000B92DB330E9F0B0FD05C0060D171D262D65
:100DE000372D06C0000F111F0250120922E030E01B
:100DF000B92DB33068F0209324013093250100937E
:100E00002001109321016092220170922301089524
:100E10000093240110932501209320013093210198
:100E20006092220170922301089560FDFECF20910F
:100E30002201220F30912301331FB72FB67021F00A
:100E40002091130130911401F894009184001091C5
:100E50008500020F131F10938900009388006160C2
:100E6000B2E0B6BB7894089560612092160120E04C
:100E700004C060612092160120E2B72FB67009F01D
:100E80006F7E789460FD05C0B0911601BB2309F018
:100E9000089501E063FF0AC0B0911401B33008F077
:100EA00002E0B0911401B63008F003E071FF01C018
:100EB00006E060FD06C0B0911601BB2311F07894E6
:100EC00008951AE083FF1AE0789400000000F89477
:100ED00062FD03C014E183FF14E171FF01C018E754
:100EE000B091B20030913901B31BB10B10F3B09146
:100EF0001601B395B0931601B5E03B2F6B2E722C03
:100F0000B0B7B072B21709F073943A95C9F77394F9
:100F10007614A8F464FFB1CF6F7E309184006090A6
:100F200085007090130180901401370D681C609249
:100F30008900309388006160B2E0B6BB9ECF64FD4B
:100F40009CCF0A9509F0B5CF7894089571FF0AC037
:100F5000B0910D01B395B0930D0160FD0CC02092CE
:100F60000D0109C060FD07C064FD05C067FD03C039
:100F7000BF91BF9114C5089520912401309125019E
:100F8000F8940091840010918500020F131F1093B4
:100F90008900009388006160B2E0B6BB7894089540
:100FA0000E94BC0700E063FF03C064FF01C001E0D2
:100FB000F89410910E01B7E01B9F212D102D78940D
:100FC000200F26951795269517952695179510931A
:100FD0000E01183718F4B8E7B0930E0100910E0116
:100FE000B0910F010B1720F060622B982C982D9870
:100FF00060FDFECF0895F8942A982898299882FFDA
:1010000007C0EFE1F1E073FF03C0B1E4BA95F1F777
:1010100095FF2A9A95FD299AB2E0B093150189C0EF
:10102000F89495FF2D9895FD2B9882FF0DC0EFE069
:10103000F1E073FF0BC0289895FF299895FD2A9839
:10104000B1E4BA95F1F702C0E9ECF0E062FF03C049
:10105000552009F02C9AB3E0B09315016AC0F894BA
:101060002A982898299882FF07C0EFEFF0E073FFD5
:1010700003C0B1E4BA95F1F795FF299A95FD2A9A34
:10108000B4E0B093150155C0F8942C9882FF0DC0C0
:10109000EFEEF0E073FF0BC095FF2A9895FD2998BD
:1010A0002898B1E4BA95F1F702C0E1ECF0E062FFF4
:1010B00006C0552021F095FF2B9A95FD2D9AB5E09D
:1010C000B093150136C0F8942A982898299882FF81
:1010D00007C0ECEDF0E073FF03C0B1E4BA95F1F79F
:1010E000289AB6E0B093150124C0F89495FF2B9888
:1010F00095FD2D9882FF10C0E2E3F1E073FF0EC072
:1011000095FF2A9895FD299895FF299895FD2A988D
:10111000B1E4BA95F1F702C0E1EDF0E062FF06C07C
:10112000552021F095FF2D9A95FD2B9AB1E0B093B3
:10113000150167FF0BC00E94A908B1E4BA95F1F749
:10114000B1E0BA95F1F72A9A289A299A6F7D789496
:10115000089520EC30E0F9012B982C982D982A98CE
:10116000289829986B7F0895ACE4B1E00FEF0D93B8
:101170000D930D930D9303E00D9304E00D930BE09D
:101180000D9301E00D9301E00D9301E00D93A8E5AF
:10119000B1E001E00D930FEF0D930D930FEF0D9361
:1011A0000D930D9303E00D9306E00D930FEF0D9358
:1011B0000D9305E20D9300ED0D930AEF0D930AEFE9
:1011C0000D9304E00D930DE00D9301E00D9300E00D
:1011D0000D930AE70D930FEF0D9301E00D93089522
:1011E00020915F0109E011E0223011F405E011E0E7
:1011F000233011F405E012E0243011F405E013E08F
:10120000253011F409E017E0263011F400E010E079
:1012100000933F0110934001209153018B7F777F12
:10122000B0915401B33019F09F7DB1FD90629F7B66
:10123000B0915501B1FD9064B22FB23011F08860C9
:1012400001C0877F0895E4E5F0E000914C010A9524
:10125000E00FF21DB491B0936D0100914D010A951C
:10126000E00FF21DB491B0936E010E94A908089599
:10127000E2E6F0E0009167010A95E00FF21DB491FB
:10128000B0936F010E94A9080895E0E7F0E0009193
:1012900052010A95E00FF21DB491B09370010E94C3
:1012A000A90808950895B09168010FEF1CE0B230CD
:1012B00011F400EA1AE0B33011F402E815E00093EB
:1012C0000F0110931001089508952091620130914B
:1012D000630197FF02C020E03FEFB32FB21B6B2EDC
:1012E000B25810F4B2E86B2E00E00395609EB12D69
:1012F000B058D8F3009347010895F894E3E0F0E084
:10130000B9E0B7BFB491B078C1F3F894A895B4B779
:10131000B070B4BFB0916000B861B0936000B0E04D
:10132000B0936000B4E0BEBFBFEFBDBF0E94A9088C
:10133000B0E0B5B9BFE3B4B9B0E0B8B9B0E0B7B99F
:10134000B0E0BBB9B0E0BAB92224A0E0B0E02D9281
:10135000AA31E9F7A0E0B1E00FEF2D920A95E9F785
:101360000E94B4080E94F30C0E94F0080E94230916
:101370000E9438090E9445090E9452090E9453099F
:101380000E9464090E94650900916401009348016C
:101390000E94A908B2E0B5BDB2E0B0938100B2E00E
:1013A000B093B100F8940E94D8030E94E3030E9416
:1013B000D4030E94E6030E94D4030E94E9030E9422
:1013C000D4030E948C0D0E94D8030E94D8030E946F
:1013D000D603B1E0B5BBB0936E00B2E0B6BBB0933C
:1013E0006F00B1E0B7BBB0937000B0917B00B06408
:1013F000B0937B00B0917A00B460B0937A000E9401
:10140000CE0378940E945C05B1E0BDBBBB27B16000
:10141000BCBB8D7F0E94D803B1E0B093090162602C
:1014200025E0B0912C01BB2309F425E00E94D003F4
:10143000B0912D01B230A0F3B92FBF7100912F01EF
:1014400000932E01B0932F01B01751F72A9549F759
:101450006D7F96FFB3E096FDB2E0B0936900BB27C5
:10146000B160BCBB8D7F0E94D6030E94D00302E016
:10147000B92FBF7109F400E0B0912D01B017A8F3A6
:10148000F8940E94E3030E94E3030E94E30378942C
:101490000E94D80320921F01B0915401B33009F487
:1014A0008DC00E94D003B0915801B13008F486C0BD
:1014B000B0910901B13008F481C0B92FBF71F1F0CA
:1014C000B0912D01BF3F08F479C0F8940E94EC035D
:1014D00078940E94D603B0912D01B130B0F7F89402
:1014E0000E94E3030E94D2030E94E30378940E94C7
:1014F000D603B0912D01BF3F90F363C3B8E09B2E9C
:101500009068F8940E94650978940E94D603F89434
:101510009F770E94650980902D01B0912D01BF3702
:10152000789408F453C00E94CE03F8940E94EC0310
:1015300078949A9429F7B82DB550B09363010E941E
:10154000D803F8940E94260D0E94920D7894BAE078
:101550009B2E9068F8940E94650978940E94D603A7
:10156000F8949F770E94650980902D01B0912D011C
:10157000BF37789460F70E94CE03F8940E94E3038B
:101580000E94D2030E94E30378949A9411F7B82D35
:10159000BB5FB09362010E94D803F8940E94260DAD
:1015A0000E94AF0D78940E94D603F8940E946509BA
:1015B0007894B0912D01BF3FB0F303C300912D018A
:1015C000B0911F010B1710F000931F010E94D6036A
:1015D00001E0B0915401B35009F405E0B0912D0140
:1015E000B01708F059CFF8940E94EC030E94EC0366
:1015F0000E94EC0378940E94D80320920901209263
:101600000A0120920B01B0910A01B395B0930A012F
:10161000BF3F79F5B0910B01B395B0930B01B09139
:10162000660109E1BA9559F002E3BA9541F00DE778
:10163000BA9529F00AEFBA9511F020920B01B091FA
:101640000B01B017B0F0B0910B01BA95B0930B013C
:10165000B4EBB0930A01B0916501B0934801F894DE
:101660000E94EC037894B0916401B09348010E9409
:10167000D6030E94D203B0910601BB2321F4B92FF7
:10168000BF7109F4CCCEB0912D01B63008F4BBCFB8
:10169000B0915401B35011F00E94D603B0910601ED
:1016A000BB2309F4BCCEF8940E94A9082092010142
:1016B0002092020120920301522C7894B0915101A2
:1016C000B09336012092170120921801209219013F
:1016D00020921A0120921B012092450160E070E0E7
:1016E00020920E010E943E06B8E0B0934501706161
:1016F0000E94CE0374FFB0E074FDB0E0B06CB09314
:101700007C00B0917A00B068B064B0937A00B09178
:101710007A00B6FDFCCF0091780010917900B0916D
:101720007A00BF77B0937A00112309F00FEF00938E
:1017300046010E94D905B8E0B093450170618090E0
:101740005301B2E0B09353010E94F008809253011C
:10175000F894BFEFB09332010E942706B0910101C7
:10176000B0933201B0933301B09334017894B1E077
:10177000B0930101B09303015B2EB0933B01B09194
:101780003101B0933A017160726020920D010E94A4
:1017900063080E9475080E9444060E943E060E944B
:1017A000A80605C00E94F008209245017F7E95FFA3
:1017B000B5E095FDB3E0B06CB0937C000E943907B2
:1017C0000E94A6070E94BC070E9471040E94D007D5
:1017D0000E94FB070E9444060E94A3060E94A806DE
:1017E0000E941507B4E0B06CB0937C000E943407EF
:1017F0000E94A6070E94BC070E9472040E94360540
:101800000E94D0070E9410080E9444060E94A3066E
:101810000E94A8060E94150795FFB3E095FDB5E06C
:10182000B06CB0937C000E9439070E94A6070E940A
:10183000BC070E9496040E94D0070E942F080E94B5
:1018400044060E94A3060E94A8060E94150795FF61
:10185000B5E095FDB3E0B06CB0937C000E94340716
:101860000E94A6070E94BC070E94D2040E94D007D3
:101870000E9444080E9444060E94A3060E94A806F3
:101880000E941507B4E0B06CB0937C000E94390749
:101890000E94A6070E94BC070E9405050E94D0076F
:1018A0000E9463080E9444060E94A3060E94A806A4
:1018B0000E94150795FFB3E095FDB5E0B06CB093BD
:1018C0007C000E94340774FFB0E074FDB0E0B06C9F
:1018D000B0937C00B0917A00B068B064B0937A00A5
:1018E0000E94A6070E94BC070E94D0070E947508AC
:1018F0000E9444060E94A3060E94A8060E94D905E1
:101900000E94150771FF25C067FD23C0B091350106
:10191000B0933201B0933301B0913101B0933A01E9
:10192000B1E0B0933B0114E624E1B0910D01B11791
:1019300050F07D7F746020930C01BFEFB0933201B3
:10194000B093330106C0B0912D01B13008F02FCF14
:1019500026C072FF10C067FD0EC0B0910C01BA9591
:1019600011F47B7F1FCFB0930C01B0912D01B130EA
:1019700008F01DCF14C0B0913001B23880F4B92FF7
:10198000BF7121F4B0910601BB2349F0B09114015D
:1019900000EF67FF01C000E6B01708F408CFF89425
:1019A0000E94A90880905301B2E0B09353010E94B5
:1019B000F0088092530120920101209202012092AE
:1019C0000301522C209236017E7F78940E94CE0330
:1019D0000E94A908B92FBF7129F4B0910601BB2359
:1019E00009F41DCD0CCEEDE0F0E00E941F0D0A358C
:1019F00009F01EC0EEE0F0E00E941F0D053A09F06C
:101A000017C03AE0ACE4B1E0E3E0F0E00E941F0D63
:101A10000D9331963A95D1F735E1A8E5B1E0EFE0C5
:101A2000F0E00E941F0D0D9331963A95D1F704C056
:101A30000E94B4080E94260DE4E2F0E00895F999AE
:101A4000FECFE1BDF2BDF89A00B508950E94490DA0
:101A50003AE0ACE4B1E0E3E0F0E00D910E94410D2A
:101A600031963A95D1F735E1A8E5B1E0EFE0F0E045
:101A70000D910E94410D31963A95D1F70E94540D77
:101A80000895F999FECF00BDE1BDF2BDFA9AF99A29
:101A90000895EDE0F0E00FEF0E94410DEEE0F0E080
:101AA0000FEF0E94410D0895EDE0F0E00AE50E947D
:101AB000410DEEE0F0E005EA0E94410D08953091FD
:101AC000490100914A01313011F400935001323044
:101AD00011F400935101333011F40093520134306A
:101AE00011F400935E01353011F400936701363034
:101AF00011F400935F01373011F400935301383033
:101B000011F400936801393011F4009354013A3014
:101B100011F400935501089525E00E94D8032A95F9
:101B2000E1F708950E94E3030E94E6030E94E9039F
:101B30000E94EC030E94D2030E94E3030E94E6038A
:101B40000E94E9030E94EC030E94D2030E94E30377
:101B50000E94E6030E94E9030E94EC0308950E949C
:101B6000EC030E94E9030E94E6030E94E3030E9443
:101B7000D2030E94EC030E94E9030E94E6030E9444
:101B8000E3030E94D2030E94EC030E94E9030E9437
:101B9000E6030E94E30308958090490190904A0172
:101BA0000E94E3030E94E3030E94E3030E94D20326
:101BB0008A94B1F70E94EC030E94D2039A94D1F761
:101BC0000895F8940E94920D78940E948C0D0E94C2
:101BD0008C0DB1E0B0934901B1E0B0934A0120927D
:101BE0004B01F8940E94CC0D7894B5E06B2E709068
:101BF0002D010E94D803B0912D017B16C1F7B130A1
:101C000018F0BF3F70F10CC00E945F0DF8940E9465
:101C1000260D0E94920DB8E0B09360000E948C0DDA
:101C20006A9429F7B0914B01B395B0934B01B3304F
:101C300008F4D7CF0E948C0DB0914A01B395B093B0
:101C40004A01F894B0914901BA95EEE7F0E0EB0F44
:101C5000F21D049178940395B0914A01B01708F4ED
:101C6000BECF0E948C0D0E948C0DB0914901B3959E
:101C7000B0934901B0914901BB3008F4ADCF0E9447
:101C8000B408F8940E94260DB8E0B09360000E945A
:021C90008C0DB9
:00000001FF
